:020000040000FA
:020000000528D1
:0800080005288316FF30850076
:1000100086018312FF308600051C1728851C3E20B0
:10002000051D5A20851D7320051EA1200C282220A5
:100030003E2022203E205A205A205A207320C220DF
:10004000A1200C28FE308600FB20FD308600FB201E
:10005000FB308600FB20F7308600FB20EF30860067
:10006000FB20DF308600FB20BF308600FB207F3086
:100070008600FB20FF308600FB2008007F308600D2
:10008000FB20BF308600FB20DF308600FB20EF30F6
:100090008600FB20F7308600FB20FB308600FB202B
:1000A000FD308600FB20FE308600FB20FF308600FE
:1000B000FB2008007E308600FB20BD308600FB2040
:1000C000DB308600FB20E7308600FB20DB3086003B
:1000D000FB20BD308600FB207E308600FB20FF30F9
:1000E0008600FB200800FE308600FB20FD308600E5
:1000F000FB20FA308600FB20F5308600FB20EA303A
:100100008600FB20D5308600FB20AA308600FB202D
:1001100055308600FB20AB308600FB205730860030
:10012000FB20AF308600FB205F308600FB20BF3015
:100130008600FB207F308600FB20FF308600FB20FE
:100140000800003086000721FF30860007210030BC
:1001500086000721FF308600072100308600072136
:10016000051CBE28FF3086000721003086000721CD
:10017000FF3086000721003086000721FF3086000F
:10018000072108007F308600FB20BF308600FB205F
:100190005F308600FB20AF308600FB2057308600A2
:1001A000FB20AB308600FB2055308600FB20AA30B8
:1001B0008600FB20D5308600FB20EA308600FB203D
:1001C000F5308600FB20FA308600FB20FD308600EB
:1001D000FB20FE308600FB20FF308600FB2008005D
:1001E00002308D00F9308C00000000008C0BF428E8
:1001F0008D0BF228080064308E00F0208E0BFD2855
:10020000080005308F00FB208F0B03290800023007
:0A02100090000121900B092908005D
:02400E00F23F7F
:00000001FF
